:020000040000FA
:04000000000E04D01A
:0800080004EF02F082AE0FD0FC
:10001000F66E040EF76E02D00CEF02F0000EF86ED2
:100020000900F53C00EF02F00900F53CFBD720EE9B
:1000300000F0700ED3129B8C82AEFED7900EAB6E8A
:10004000260EAC6EB886020ED56EAB98AE50AE5092
:10005000D76AD66AF2944ED8D58E4CD8D59EF2B4D3
:10006000F7D7D6CFAFFFD7CFB0FFAB8822D90F0AD3
:10007000ECE10F0E19D900EE04F01BD90F0AF9E0DC
:100080000250040A07E00250050A01E112D902C039
:10009000ECFFF3D710EE05F0006A016AEDCFF4FF34
:1000A000E65030D8E250EA62FBD7E150E962F8D777
:1000B0000150F462CAD70050EF62C7D7006A016AE4
:1000C0000650F66EA96E0750F76EAA6E08C0F8FFCC
:1000D00000EE0BF00A0E0560B8D7F9500544F9267A
:1000E00027D02FD039D04FD07CD0A9D0B6D0C5D012
:1000F00099D7FF000400F2B4120082BEFCD782AE92
:10010000FED71200011800C001F0006EE83A0F0B94
:10011000001A0038F00B011A0038E844011AE00B0D
:10012000011A001A120000030105FF8400000000FC
:10013000260EF66E010EF76E000EF86E0A0E0A6EAF
:100140000B6A0900F550A4D8DDDF0A06000E0B5A31
:100150000A500B10F6E195D00900F550D3DFF650A8
:100160003F0BFAE1005048EC01F0015048EC01F07F
:100170000A06000E0B5A0A500B10EEE186D0FF0063
:10018000FF00FF00FF00C00EF616000EF65C000E2A
:10019000F758010EF85802E6A66A17D0000EF65C72
:1001A000000EF758000EF8580DE6000EF65C030E30
:1001B000F758000EF85806E7A66A07D0FF00FF00C0
:1001C000FF00FF00940EA66E82D8400EF65EE86A2D
:1001D000F75AF85A0A2ED7D750D0FF00FF00FF0079
:1001E000FF00C00EF616000EF65C000EF758010E6A
:1001F000F85802E6A66A16D0000EF65C000EF75814
:10020000000EF8580DE6000EF65C030EF758000ECF
:10021000F85806E7A66A06D0FF00FF00FF00FF00BF
:10022000840EA66EEECFF5FF0C000900F6503F0BD2
:10023000F9E10A004CD809000A2ED3D71ED0A66ACD
:10024000A680A850A94AAA2A23D85CDF0A06000E75
:100250000B5A0A500B10F4E114D0040EA66EECCF2A
:10026000A8FF35D8A6B2FED7A94AAA2A0A06000EC8
:100270000B5A0A500B10F3E100D0A66A055008D8BB
:1002800041DF005005D8015003D8040E0DD8EED63A
:10029000036E0F0A06E00350040A03E00350050A48
:1002A00002E1050E01D8035004009EA8FED7AD6EF2
:1002B0001200ABB2FF0004009EAAFDD7AE50026E42
:1002C0001200FF00FF00FF00A66AF56E0C0004009C
:0E02D000550EA76EAA0EA76EA68200001200A1
:020000040030CA
:03000100021F1EBD
:020005008381F5
:060008000FC00FE00F40E5
:00000001FF
